:100000000C94DA040C941E050C941E050C941E0529
:100010000C941E050C941E050C941E050C941E05D4
:100020000C941E050C941E050C94B7180C94891999
:100030000C94EC270C941E050C941E050C941E05C4
:100040000C941E050C941E050C941E050C941E05A4
:100050000C941E050C9454280C941E050C941E053B
:100060000C941E050C941E050C941E050C941E0584
:100070000C941E050C941E050C941E050C941E0574
:100080000C94AD0E0C941E050C941E050C941E05CC
:100090000C941E050C941E050C941E050C941E0554
:1000A0000C941E050C941E050C941E0579058905FB
:1000B0009B05AB05B105C005CC05D205E005E905FA
:1000C000FA050A0610064006F619181A061B181A31
:1000D000061B5D1A801A061BD51AE81AEB1DEB1DCC
:1000E000281E281E821EC01E38213821D91E382104
:1000F000DA1FDA1F9D20B4203821232107634236FE
:10010000B79BD8A71A39685618AEBAAB558C1D3CA8
:10011000B7CC5763BD6DEDFD753EF6177231BF006C
:100120000000803F08000000BE922449123EABAAA6
:10013000AA2ABECDCCCC4C3E00000080BEABAAAA01
:10014000AA3E00000000BF000000803F0000000049
:1001500000084178D3BB4387D1133D190E3CC3BD82
:100160004282AD2B3E68EC8276BED98FE1A93E4C2F
:1001700080EFFFBE01C4FF7F3F00000000002B00A6
:1001800014001A000800150017001C0018000C00CD
:10019000120013002A0029000400160007000900BD
:1001A0000A000B000D000E000F0033003400E100C8
:1001B0001D001B000600190005001100100036008C
:1001C0003700380028000530E000E200E30003308B
:1001D0002C002C0004305000510052004F002B0026
:1001E00014001A00090013000A000D000F00180087
:1001F0001C0033002A002900040015001600170017
:1002000007000B00110008000C0012003400E10090
:100210001D001B000600190005000E00100036002E
:100220003700380028000530E000E200E30003302A
:100230002C002C0004305000510052004F002B00C5
:1002400034003600370013001C0009000A000600C5
:1002500015000F002A0029000400120008001800F1
:100260000C0007000B001700110016003800E10019
:10027000330014000D000E001B00050010001A00D2
:1002800019001D0028000530E000E200E300033003
:100290002C002C0004305000510052004F00350259
:1002A0001E021F0220022102220223022402250232
:1002B000260227022A004C003A003B003C003D0089
:1002C0003E003F002D022E022F02300231020100BB
:1002D000400041004200430044004500010001008D
:1002E0000100010001000100010001000100010006
:1002F000010001000100AB00AA00A900AE0035001A
:100300001E001F00200021002200230024002500E1
:10031000260027002A004C003A003B003C003D002C
:100320003E003F002D002E002F0030003100010064
:10033000400041004200430044004500010001002C
:1003400001000100010001000100010001000100A5
:10035000010001000100AB00AA00A900AE000000EE
:10036000000000000000000000000000000000008D
:10037000000000000000000000000000000000007D
:10038000000000000000000000000000000000006D
:10039000000000000000000000000000000000005D
:1003A000000000000000000000000000000003301A
:1003B00000000000043000000000000000001E00EB
:1003C0001E001E001E001E001E001E001E001E003D
:1003D0001E001E001E00000014001A000800150078
:1003E00017001C0018000C00120013002F00000062
:1003F00004001600070009000A000B000D000E00A3
:100400000F00330034000D3000000000060019001A
:1004100000000000110010000000000000000000BB
:1004200000000000000000000000000000000000CC
:1004300000000000000000000000000000000000BC
:1004400000000000000000000000000000000000AC
:10045000000000000000000000000000000000009C
:100770000000000000000000000000000000010078
:100780000050010001000100010001000100010012
:10079000010001004C00010001000100073006309B
:1007A000135012500030013002300C3001000100B3
:1007B0000B300A300930083001000100010001004F
:1007C0000100010001000100010001000100010021
:1007D00001000100010001000100010001002803E7
:1007E000540068006500200050006C0061006E003D
:1007F00063006B0020004B006500790062006F0011
:1008000061007200640000002C034F00720074004D
:1008100068006F006C0069006E0065006100720086
:1008200020004B006500790062006F0061007200DB
:100830006400730000000403090409026D00040150
:1008400000A0FA09040000010301010009211101BF
:100850000001223F000705810308000A0904010086
:100860000103010200092111010001224D000705C9
:10087000820308000A0904020001030000000921A4
:10088000110100012236000705830308000A09044C
:1008900003000103000000092111010001223900B9
:1008A000070584031000011201100100000008ED8B
:1008B000FE606001000102000105010906A10105B9
:1008C0000719E029E7150025019508750181020542
:1008D0000819012905950575019102950175039186
:1008E0000105071900297715002501957875018103
:1008F00002C005010980A101850216010026B7008A
:100900001A01002AB700751095018100C0050C0975
:1009100001A1018503160100269C021A01002A9CF0
:1009200002751095018100C005010902A1010901AC
:10093000A100050919012905150025019505750175
:100940008102950175038101050109300931158185
:10095000257F95027508810609381581257F950147
:1009600075088106050C0A38021581257F950175E9
:10097000088106C0C005010906A101050719E02983
:10098000E71500250195087501810295017508811B
:100990000105081901290595057501910295017553
:1009A0000391010507190029FF150025FF9506751C
:1009B000088100C011241FBECFEFDAE0DEBFCDBF3B
:1009C00004B603FE24C08091690490916A04A0914A
:1009D0006B04B0916C048730904BA740B04BB9F4D6
:1009E0001092690410926A0410926B0410926C04C5
:1009F00014BE84B7877F84BF88E10FB6F8948093D4
:100A00006000109260000FBEE0E0F8E3099513E08B
:100A1000A0E0B1E0E2E4F4E602C005900D92A23657
:100A2000B107D9F714E0A2E6B3E001C01D92A936E0
:100A3000B107E1F70E94FD150C941F320C940000E1
:100A4000279A2F988FEF9FEF9093870080938600CF
:100A50008AE08093800089E1809381000C94562D78
:100A6000282F81110BC080918000877F80938000A8
:100A700010928D0010928C002F9808952F988091DD
:100A80008000886080938000233019F48FEF9FEFFF
:100A90000FC083E090E0821B9109880F991F2FEF10
:100AA0003FEFA90102C0569547958A95E2F7CA0122
:100AB00090938D0080938C000895CF93DF93EC0189
:100AC0000E94ED28BE0180E090E0DF91CF910C9470
:100AD00018250F931F93462F50E04E30510508F014
:100AE000DEC0DC01FA01EA5AFF4F12968C910C9499
:100AF000E331882309F4D3C000E010E0980140E01E
:100B000064E070E089E292E00E942B1281E090E0C4
:100B10000FC0882309F4C3C000E010E0980140E052
:100B200066E070E089EB91E00E942B1282E090E099
:100B30000E945D05B4C0882309F4B1C000E010E054
:100B4000980140E068E070E089EE91E00E942B128D
:100B500084E090E0EDCF882311F083E005C083E0CE
:100B60000CC0882349F084E00E94952540E164E0B0
:100B700083E00E946D0A93C084E00E94B625F6CF00
:100B8000882331F085EE0E947F1C0E94AD2D87C026
:100B900085EE0E94471D83C0882309F480C00E940F
:100BA000BF0D7DC0882309F47AC00E94B80D00E013
:100BB00010E0980140E065E070E089E492E027C031
:100BC000882309F46CC085E00E94B6250E94E00DE0
:100BD00066C0882309F463C000E010E0980140E09B
:100BE00068E070E089E191E00E942B1285E00E94AC
:100BF000952555C0882309F452C00E94BE1200E01A
:100C000010E0980140E068E070E089E191E00E9426
:100C10002B1245C0882309F442C00E94C912EFCFAD
:100C20008823E9F100E010E0980140E066E070E020
:100C300089E891E00E942B1284E00E94B62583E0AF
:100C40000E94B62580E10E94B62585E00E94B62567
:100C50000E94E00D86E00E9495250E94DA2881110D
:100C600002C00E94B6280E94F22890E09093680487
:100C7000809367048068809367040E94F6280FC001
:100C8000882369F000E010E0980140E066E070E041
:100C900089E591E00E942B1286E00E94B62580E053
:100CA00090E01F910F9108950F931F932FEF89EFFD
:100CB00090E0215080409040E1F700C0000000E04B
:100CC00010E0980140E065E070E089E492E00E9465
:100CD0002B121F910F9108950F931F9300E010E0C6
:100CE000980140E063E070E081E091E00E942B1207
:100CF0002FEF82E597E0215080409040E1F700C05F
:100D000000001F910F910895CF92DF92EF92FF9212
:100D10000F931F93CF93DF93CDB7DEB7CC58D10994
:100D20000FB6F894DEBF0FBECDBF2091210425FF82
:100D3000C5C08C01FC01928180910001992309F4C6
:100D400060C096E4EEE8F2E0DE01A95BBF4F0190DF
:100D50000D929A95E1F7F8019081E0916203F0918C
:100D60006303E90FF11DEE0FFF1F27E430E02C0FA6
:100D70003D1FE20FF31F60817181680F711D88278D
:100D800077FD8095982F0E94F12E20E030E040E41E
:100D900051E40E94562E6B017C01F801218184E010
:100DA00090E0821B9109BC01882777FD8095982FE0
:100DB0000E94F12E9B01AC01C701B6010E94EE2DED
:100DC0009B01AC0160E070E080E090E40E94643040
:100DD00020E030E04CE551E40E9401304FE050E06B
:100DE000C457DF4F0FB6F894DEBF0FBECDBFDF9103
:100DF000CF911F910F91FF90EF90DF90CF900C94C7
:100E0000CB1196E4EEE8F2E0DE01119601900D922E
:100E10009A95E1F7F8019081E0916203F091630304
:100E2000E90FF11DEE0FFF1F21E030E02C0F3D1FF9
:100E3000E20FF31F60817181680F711D882777FDB4
:100E40008095982F0E94F12E20E030E040E451E49C
:100E50000E94562E6B017C01F801218184E090E014
:100E6000821B9109BC01882777FD8095982F0E94ED
:100E7000F12E9B01AC01C701B6010E94EE2D9B0132
:100E8000AC0160E070E080E090E40E94643020E01B
:100E900030E04CE551E40E940130C457DF4F0FB6FB
:100EA000F894DEBF0FBECDBFDF91CF911F910F91A0
:100EB000FF90EF90DF90CF900C94130EC457DF4F4C
:100EC0000FB6F894DEBF0FBECDBFDF91CF911F915B
:100ED0000F91FF90EF90DF90CF90089508950E94BA
:100EE00020056E9A769A0C9454060C946E070C9416
:100EF00084060895880F991FFC01E250F040859107
:100F000094910895880F991FFC01E258FE4F859136
:100F1000949108950F931F93CF93DF93EC01811564
:100F200020E49207A0F5C11580E3D80708F0E1C0DE
:100F3000C83ED105D8F4C03ED10508F0EEC1C83A8C
:100F4000D10578F4C53AD10508F074C0C130D10597
:100F500009F46DC008F4DEC1C430D10508F0DDC16C
:100F6000D9C1CB3BD10508F470C0D4C1C11590E202
:100F7000D90708F0B9C0C11521E0D20708F0CDC1EA
:100F8000C03FD10508F4C6C18E01106506C2C1304C
:100F900080E5D80709F4BDC068F5C13120E4D20767
:100FA00009F4AEC050F4C03190E4D90708F0A5C0F0
:100FB000CF70DD278E01146DF0C1C33120E4D2075C
:100FC00009F4A4C008F49FC0C115D04509F0A2C11E
:100FD0000E945C210E94E00D0E946C069FEF24E3BA
:100FE0008CE0915020408040E1F700C000000E945A
:100FF0007928D3C1C11520E6D20730F4C11581E5A7
:10100000D80708F48CC02DC1C11590E7D90708F4A2
:1010100081C1C11520E8D20708F478C1C11580E963
:10102000D80708F077C1DF708E01106AB6C101E001
:1010300010E0B3C1C53AD10509F471C1C63AD10572
:1010400009F070C102E810E4A8C1C83AD10509F45A
:101050006CC1C93AD10509F46BC1CA3AD10509F48A
:101060006AC1CB3AD10509F469C1CC3AD10509F47A
:1010700068C1CD3AD10509F467C1C03BD10509F477
:1010800066C1CE3AD10509F465C1CF3AD10509F45C
:1010900064C1C13BD10509F463C1C23BD10509F468
:1010A00062C1C33BD10509F461C1C43BD10509F458
:1010B00060C1C53BD10509F45FC1C63BD10509F448
:1010C0005EC1C73BD10509F45DC1C83BD10509F438
:1010D0005CC1C93BD10509F45BC1CA3BD10509F428
:1010E0005AC100E014E459C1CE019F700E948207EA
:1010F00055C1DD278E01106C50C100E011ED4DC1CE
:1011000000E010ED4AC100E012ED47C100E013ED30
:1011100044C180913D04816080933D043EC10E94A2
:10112000DA28811102C00E94B6280E94F22890E0BD
:101130009093680480936704C23090E5D90721F446
:1011400080916704816086C0C43020E5D20721F415
:101150008091670482607EC0C63080E5D80721F4A4
:1011600080916704846076C0C83090E5D90719F48F
:101170008091670427C0CA3020E5D20721F480910E
:101180006704806167C0CC3080E5D80721F4809186
:10119000670480625FC0CE3090E5D90721F480916A
:1011A0006704806457C0C03120E5D20721F48091E4
:1011B000670480684FC0C23180E5D80729F4809168
:1011C00067048460886046C0C33090E5D90721F485
:1011D000809167048E7F3EC0C53020E5D20721F4A0
:1011E000809167048D7F36C0C73080E5D80721F431
:1011F000809167048B7F2EC0C93090E5D90719F420
:101200008091670426C0CB3020E5D20721F480917D
:1012100067048F7E1FC0CD3080E5D80721F4809110
:1012200067048F7D17C0CF3090E5D90721F48091F6
:1012300067048F7B0FC0C13120E5D20721F4809174
:1012400067048F7707C0C331D04531F480916704BC
:101250008B7F877F80936704809167040E94F628C4
:101260009CC08D2F99278F70992781309105D9F4D3
:101270009E012370332702C0880F991F2A95E2F739
:101280009C688E0144E0000F111F4A95E1F700278A
:101290001370802B912B53E0CC0FDD1F5A95E1F793
:1012A000C076DD272FC08230910531F4DC2FCC27AA
:1012B0008E01016F106A71C08330910569F4CE010F
:1012C0008370992701E010E002C0000F111F8A957A
:1012D000E2F7C8019C680FC0049709F05EC0CE0118
:1012E0008370992701E010E002C0000F111F8A955A
:1012F000E2F7C8019A6823E0CC0FDD1F2A95E1F7D9
:10130000C07ED7708C010C2B1D2B47C0DF708E0167
:10131000106243C000E010E040C08E013EC001E812
:1013200010E43BC003E810E438C002EE14E435C01A
:1013300009EE14E432C00AEE14E42FC005EB14E405
:101340002CC006EB14E429C007EB14E426C00CEC17
:1013500014E423C00DEC14E420C003E815E41DC020
:101360000AE815E41AC002E915E417C004E915E417
:1013700014C001E216E411C003E216E40EC004E258
:1013800016E40BC005E216E408C006E216E405C048
:1013900007E216E402C00AE216E4C801DF91CF9129
:1013A0001F910F9108959CE0799FF001112490E323
:1013B000899FE00DF11D1124E60FF11DEE0FFF1FB7
:1013C000E258FE4F85919491803E9105E0F4803C77
:1013D000910558F58133910509F46FC048F48932BD
:1013E000910509F463C08A32910509F46DC072C099
:1013F00089339105E9F082389105D1F08533910563
:1014000009F44DC067C0833E910581F138F4803EF8
:101410009105B9F0823E9105D9F05CC0863E9105F8
:1014200061F1873E9105A1F155C00E947A070895A8
:101430002091670420FD02C021FF4CC080EE90E0A7
:1014400049C08091670480FFF9CF89E390E042C0F2
:101450008091670482FF0EC08091670484FF03C0FF
:1014600080E090E037C083EE90E034C08091670464
:1014700082FFF2CF82EE90E02DC08091670483FF5F
:101480000BC08091670484FDEBCF87EE90E022C013
:101490008091670483FFF5CF86EE90E01BC08091BA
:1014A000670485FF07C089E290E014C0809167045B
:1014B00085FFF9CF85E390E00DC08091670486FF3A
:1014C00007C08AE290E006C08091670486FFF9CFEA
:1014D00081E390E00E948A070895CF92DF92EF9215
:1014E000FF920F931F9301E010E020E030E06801CD
:1014F000790104C0CC0CDD1CEE1CFF1C8A95D2F7D0
:1015000004C0000F111F221F331F6A95D2F70C2948
:101510001D292E293F29C0902104D0902204E0905B
:101520002304F0902404C022D122E222F322842F4B
:10153000C016D106E206F30641F41F910F91FF9009
:10154000EF90DF90CF900C9495251F910F91FF9015
:10155000EF90DF90CF900C94B62508950C94AD0ACF
:101560005F926F927F928F929F92AF92BF92CF9233
:10157000DF92EF92FF920F931F93CF93DF93CDB73C
:10158000DEB728970FB6F894DEBF0FBECDBFCE01F1
:1015900001966C014E0199E0890E911C20E030E02B
:1015A00040E050E060E070E000E010E0E12CF12C61
:1015B0006C2C5D2C88E0782EAA24A394B12CE4ED49
:1015C000F2E0A62DB52D872D01900D928A95E1F7B9
:1015D000F601819191916F01FC01E07FFF27E032DC
:1015E000F10559F48F709927F50102C0EE0FFF1F26
:1015F0008A95E2F7EE2AFF2A37C0E033F10559F465
:101600008F709927F50102C0EE0FFF1F8A95E2F750
:101610000E2B1F2B29C0E034F10559F48F70992748
:10162000F50102C0EE0FFF1F8A95E2F76E2B7F2BAC
:101630001BC0E035F10559F48F709927F50102C000
:10164000EE0FFF1F8A95E2F74E2B5F2B0DC0E036A1
:10165000F10551F48F709927F50102C0EE0FFF1FBD
:101660008A95E2F72E2B3F2BC814D90409F0A7CF97
:1016700084B19E2D9095892384B985B1E82AE5B877
:1016800087B1902F9095892387B988B1082B08B925
:101690008AB1962F909589238AB98BB1682B6BB943
:1016A0008DB1942F909589238DB98EB1482B4EB969
:1016B00080B3922F9095892380BB81B3282B21BBC7
:1016C00028960FB6F894DEBF0FBECDBFDF91CF9145
:1016D0001F910F91FF90EF90DF90CF90BF90AF9050
:1016E0009F908F907F906F905F9008955F926F9220
:1016F0007F928F929F92AF92BF92CF92DF92EF92A2
:10170000FF920F931F93CF93DF93CDB7DEB7689708
:101710000FB6F894DEBF0FBECDBF85B7806885BF1A
:1017200085B7806885BF0E94B00ACE0101966C0122
:101730004E0199E1890E911C20E030E040E050E03C
:1017400060E070E000E010E0E12CF12C6C2C5D2CEE
:1017500088E1782EAA24A394B12CECEDF2E0A62D1A
:10176000B52D872D01900D928A95E1F7F6018191B3
:1017700091916F01FC01E07FFF27E032F10559F400
:101780008F709927F50102C0EE0FFF1F8A95E2F7CF
:10179000EE2AFF2A37C0E033F10559F48F709927FC
:1017A000F50102C0EE0FFF1F8A95E2F70E2B1F2BEB
:1017B00029C0E034F10559F48F709927F50102C072
:1017C000EE0FFF1F8A95E2F76E2B7F2B1BC0E035D3
:1017D000F10559F48F709927F50102C0EE0FFF1F34
:1017E0008A95E2F74E2B5F2B0DC0E036F10551F4E0
:1017F0008F709927F50102C0EE0FFF1F8A95E2F75F
:101800002E2B3F2BC814D90409F0A7CF84B19E2DED
:101810009095892384B985B1E82AE5B887B1902FDE
:101820009095892387B988B1082B08B98AB1962F7A
:10183000909589238AB98BB1682B6BB98DB1942FA0
:10184000909589238DB98EB1482B4EB980B3922FD4
:101850009095892380BB81B3282B21BB10926D0307
:1018600010926C03109265031092640310926F0340
:1018700010926E0310926703109266031092710328
:101880001092700310926903109268031092730310
:101890001092720310926B0310926A0368960FB64F
:1018A000F894DEBF0FBECDBFDF91CF911F910F9196
:1018B000FF90EF90DF90CF90BF90AF909F908F9070
:1018C0007F906F905F900C946F077F928F929F92A2
:1018D000AF92BF92CF92DF92EF92FF920F931F933E
:1018E000CF93DF93CDB7DEB7A0970FB6F894DEBFE6
:1018F0000FBECDBF6E0149E1C40ED11C84E6E82EB7
:1019000083E0F82E98E0792EBC2CAD2C01E010E09D
:1019100028E1822E35E0932EE4EDF2E0AB2DBA2DD6
:10192000872D01900D928A95E1F7F60181919191B1
:101930006F019C01207F33272032310591F424B1BF
:101940008F709927A80102C0440F551F8A95E2F7AE
:10195000CA01922F982B94B995B18095892385B9A6
:1019600053C02033310591F427B18F709927F801C6
:1019700002C0EE0FFF1F8A95E2F7CF01922F982B3E
:1019800097B998B18095892388B93EC02034310534
:1019900091F42AB18F709927A80102C0440F551FF6
:1019A0008A95E2F7CA01922F982B9AB99BB180953C
:1019B00089238BB929C02035310591F42DB18F7061
:1019C0009927F80102C0EE0FFF1F8A95E2F7CF01B9
:1019D000922F982B9DB99EB1809589238EB914C002
:1019E0002036310589F420B38F709927A80102C0F1
:1019F000440F551F8A95E2F7CA01922F982B90BB8E
:101A000091B38095892381BB50EA5A95F1F7BE01C5
:101A10006F5F7F4F20E030E040E050E0ECEDF2E01F
:101A2000DE011196882D01900D928A95E1F7FB0158
:101A300081919191BF01FC01E07FFF27E032F10528
:101A400011F4E3B113C0E033F10511F4E6B10EC0B7
:101A5000E034F10511F4E9B109C0E035F10511F404
:101A6000ECB104C0E036F105B9F4EFB1F0E08F70ED
:101A7000992702C0F595E7958A95E2F7E0FD08C041
:101A8000C801042E02C0880F991F0A94E2F702C011
:101A900080E090E0282B392B4F5F5F4F4C30510591
:101AA00009F0BCCFF701808191818217930721F063
:101AB00031832083909271020E94B00AF2E0EF0E0F
:101AC000F11C4CE6E41643E0F40609F025CF8091C2
:101AD0007102882361F1815080937102882339F06B
:101AE0008FE99FE00197F1F700C0000020C08091CE
:101AF00064039091650390936D0380936C038091D0
:101B000066039091670390936F0380936E038091B7
:101B1000680390916903909371038093700380919F
:101B20006A0390916B0390937303809372030E94F6
:101B3000750781E0A0960FB6F894DEBF0FBECDBF4B
:101B4000DF91CF911F910F91FF90EF90DF90CF9099
:101B5000BF90AF909F908F907F900895E82FF0E016
:101B6000EE0FFF1FE459FC4F808191810895089585
:101B7000809152048160809352040C9408298091D2
:101B800052048E7F809352040C9408290E94DA2814
:101B9000811102C00E94B6280E9404298093520439
:101BA0003E9A809171008D7F8093710082E08093D6
:101BB00090008AE18093910081E0809376030895FC
:101BC00080917603811102C00E94C60D1092C60357
:101BD0001092C503809171008D7F80937100809178
:101BE00090008F7780939000109288031092870363
:101BF0001092BF031092C0031092C1031092C2034F
:101C00001092BE031092BD03EDE9F3E0ADE8B3E03E
:101C100011921192119211921D921D9283E0ED3B4F
:101C2000F807B1F70895CF92DF92EF92FF920F93EA
:101C30001F93CF93DF9320918703222309F484C05D
:101C40006B017C0180917603811102C00E94C60D58
:101C50000DEB13E0C7E0D0E0A7019601F8019291E7
:101C60008291729162918F010E94522E811131C036
:101C7000FE01EE0FFF1FEE0FFF1FE356FC4F108219
:101C8000118212821382DE01AA0FBB1FA357BC4F21
:101C900011961C921E92C730D105E9F0219644811D
:101CA0005581668177814083518362837383148277
:101CB00015821682178212968D919C911397119618
:101CC0009C938E9313961C921E92129734961296A2
:101CD000E2CF219708F68091C5039091C603019742
:101CE00097FD05C09093C6038093C50304C010926E
:101CF000C6031092C5038091C5039091C60320913D
:101D0000C3033091C4032817390724F01092C40389
:101D10001092C303892BC1F4809171008D7F809351
:101D20007100809190008F77809390001092BF0394
:101D30001092C0031092C1031092C2031092BE030E
:101D40001092BD0310928703DF91CF911F910F91E5
:101D5000FF90EF90DF90CF9008951F920F920FB6F3
:101D60000F9211244F925F926F927F928F929F9267
:101D7000AF92BF92CF92DF92EF92FF922F933F9359
:101D80004F935F936F937F938F939F93AF93BF9383
:101D9000CF93DF93EF93FF9380918703882309F418
:101DA0009BC1C091C503D091C6031C161D060CF043
:101DB00093C14090770350907803609079037090BE
:101DC0007A0320E030E0A901C301B2010E94FD2F97
:101DD00018160CF065C0C130D10509F452C08091CD
:101DE000C3039091C403BE010E94CF317C01909344
:101DF000C4038093C3038090890390908A03A090CA
:101E00008B03B0908C0320E030E040E85FE3C50135
:101E1000B4010E94EE2D6093890370938A0380932E
:101E20008B0390938C03F701EE0FFF1FEE0FFF1F44
:101E3000E356FC4FA30192016081718182819381FD
:101E40000E94562E20E030E040E05EE30E94013028
:101E50009B01AC01C501B4010E94FD2F18168CF442
:101E6000C7010196BE010E94CF319093C4038093B5
:101E7000C3031092890310928A0310928B0310926D
:101E80008C03E091C303F091C403EE0FFF1FEE0F2C
:101E9000FF1FE356FC4F6081718182819381D0C026
:101EA000C090BF03D090C003E090C103F090C20384
:101EB00020E030E0A901C701B6010E94522E21970F
:101EC000882309F4A2C0FE01EE0FFF1FEE0FFF1FD3
:101ED000E356FC4F80809180A280B380A5019401DD
:101EE000C701B6010E94522E87FF31C0A50194019F
:101EF00060E070E08CED93EC0E94562E20E030E024
:101F000040E451E40E94562E20E030E040E05FE3E0
:101F10000E9401309B01AC0160E070E080E090E441
:101F20000E9464309B01AC01C501B4010E940130E4
:101F30009B01AC01C701B6010E94522E87FF07C06A
:101F4000A701960160E070E08CED93E439C0A50133
:101F50009401C701B6010E94FD2F18160CF055C060
:101F6000A501940160E070E08CED93E40E94562E90
:101F700020E030E040E451E40E94562E20E030E0C2
:101F800040E05FE30E9401309B01AC0160E070E043
:101F900080E090E40E9464309B01AC01C501B40173
:101FA0000E9401309B01AC01C701B6010E94FD2FC8
:101FB00018165CF5A701960160E070E08CED93ECDB
:101FC0000E94562E20E030E040E451E40E94562E5C
:101FD00020E030E040E05FE30E9401309B01AC0173
:101FE00060E070E080E090E40E9464309B01AC010E
:101FF000C701B6010E9401306093BF037093C00314
:102000008093C1039093C20313C0FE01EE0FFF1F24
:10201000EE0FFF1FE356FC4F80819181A281B381B7
:102020008093BF039093C003A093C103B093C203F6
:102030006091BF037091C0038091C1039091C2036E
:1020400020917403309175032F3F4FEF340731F027
:102050002F5F3F4F30937503209374030E94D41277
:102060006B017C0120E034E244EF51E40E94522EE7
:1020700087FF08C086EFC82E88E2D82E84EFE82EAE
:1020800081E4F82E20E030E040E051E4C701B601E1
:102090000E9401309B01AC0160E074E284E79BE4A4
:1020A0000E94562E6B017C010E94BE2E70939700F9
:1020B00060939600209172023091730240917402F5
:1020C00050917502C701B6010E9401300E94BE2ED8
:1020D000709399006093980080918803882309F495
:1020E00033C1C0908303D0908403E0908503F090C7
:1020F000860320E030E0A901C701B6010E94FD2F50
:102100001816D4F580917403909175038F3F2FEFCB
:10211000920729F001969093750380937403C70189
:10212000B6010E94D41220E030E040E051E40E9469
:1021300001309B01AC0160E074E284E79BE40E9403
:10214000562E6B017C010E94BE2E70939700609307
:102150009600209172023091730240917402509166
:102160007502C701B6010E9401300E94BE2E709315
:1021700099006093980008C0109297001092960002
:10218000109299001092980060917D0370917E03E7
:102190006F5F7F4F70937E0360937D032091960065
:1021A0003091970080E090E0232BF1F0C0919600F1
:1021B000D09197000E94EF2E6B017C01BE0180E060
:1021C00090E00E94EF2E9B01AC0160917F03709123
:1021D000800380918103909182030E94562E20E01B
:1021E0003FEF4FE757E410C00E94EF2E6B017C01D8
:1021F00020E030EE4FEF54E460917F037091800354
:1022000080918103909182030E9401309B01AC0177
:10221000C701B6010E94FD2F87FD96C080917B0308
:102220008F5F80937B0390E020914E0430914F04A8
:1022300082179307A0F080915904882319F0109217
:102240007B030DC0809171008D7F80937100809120
:1022500090008F7780939000109288037DC08091CA
:102260007C03C0917B03811128C0C0905304D0909F
:102270005404E0905504F090560420E030E0A901A9
:10228000C701B6010E94FD2F1816BCF481E08093AF
:102290007C031092830310928403109285031092A2
:1022A0008603C0927F03D0928003E0928103F09274
:1022B0008203C150C0937B0343C010927C031092F1
:1022C000750310927403E0915004F091510448E0BA
:1022D000C49FE00DF11D112480819181A281B38101
:1022E0008093830390938403A0938503B093860324
:1022F00020E030E040E85EE364817581868197816B
:102300000E9401306B017C0120E030E048EC52E497
:1023100060917602709177028091780290917902B3
:102320000E94562E9B01AC01C701B6010E940130EC
:1023300060937F0370938003809381039093820363
:1023400010927E0310927D038091520480FD04C0A0
:102350001092880310928703FF91EF91DF91CF9144
:10236000BF91AF919F918F917F916F915F914F91AD
:102370003F912F91FF90EF90DF90CF90BF90AF9063
:102380009F908F907F906F905F904F900F900FBEB7
:102390000F901F901895CF92DF92EF92FF92CF93FC
:1023A000DF936B017C01EA0180917603811102C009
:1023B0000E94C60D8091520480FF46C08091C503E3
:1023C0009091C60308970CF03FC0809171008D7FFB
:1023D000809371008091880381110E94E00D81E05B
:1023E00080938703109275031092740320E030E00D
:1023F000A901C701B6010E94FD2F1816DCF48091D7
:10240000C5039091C603FC01EE0FFF1FEE0FFF1FE7
:10241000E356FC4FC082D182E282F382FC01EE0FD0
:10242000FF1FE357FC4FD183C08301969093C603EF
:102430008093C503809171008260809371008091C8
:102440009000806880939000DF91CF91FF90EF9093
:10245000DF90CF9008958F929F92AF92BF92CF92CC
:10246000DF92EF92FF920F931F93CF93DF93EC01D4
:102470007B01D42E4801590180917603811102C05D
:102480000E94C60D8091520480FF6BC08091710044
:102490008D7F809371008091870381110E94E00DF0
:1024A00081E080938803D0935104C0935004F0924C
:1024B0004F04E0924E04D0925904809253049092BB
:1024C0005404A0925504B0925604109289031092BD
:1024D0008A0310928B0310928C0310927B038881E5
:1024E0009981AA81BB818093830390938403A093F5
:1024F0008503B093860320E030E040E85EE36C8122
:102500007D818E819F810E9401306B017C0120E0E2
:1025100030E048EC52E4609176027091770280914D
:102520007802909179020E94562E9B01AC01C7015E
:10253000B6010E94013060937F0370938003809303
:1025400081039093820310927E0310927D03809109
:102550007100826080937100809190008068809308
:102560009000DF91CF911F910F91FF90EF90DF903E
:10257000CF90BF90AF909F908F9008958091C703A8
:1025800090E0019666E070E00E94CF318093C7032F
:1025900008958091C70390E0019766E070E00E9483
:1025A000CF318093C70308958F929F92AF92BF92CD
:1025B000CF92DF92EF92FF920F931F93CF93DF930F
:1025C0006B017C01C0917403D0917503BE0180E062
:1025D00090E00E94EF2E4B015C01A701960160E0A4
:1025E00070E08CE594E40E94562E9B01AC01C5017D
:1025F000B4010E9401300E94C32E2091C7032330F2
:1026000009F473C028F4222351F02130E9F02CC1E1
:10261000243009F4A0C0253009F4E0C025C180E0D1
:1026200090E0A0E0BFE38093720290937302A093C6
:102630007402B0937502109277031092780310928F
:10264000790310927A0310C11092770310927803E5
:102650001092790310927A036431710540F46A3064
:10266000710560F520E030E040E85EE32BC0693C96
:10267000710508F0AAC080E090E00E94EF2E20E0F3
:1026800030E040EA51E40E94ED2D20E030E044E3E8
:1026900053E40E94562E9B01AC010E94013020E0C1
:1026A00030E040E05EE30E9401309B01AC0160E05D
:1026B00070E080E09EE30E94ED2D44C020E030E019
:1026C00040E05FE3C701B6010E9401306B017C016D
:1026D00080E090E0A0E0BEE38093720290937302EA
:1026E000A0937402B0937502BFC01092770310924A
:1026F00078031092790310927A034AE0469F900182
:10270000479F300D1124C90168EB7BE00E94BB316B
:10271000BC016C5D754077FF03C0719561957109CF
:10272000882777FD8095982F0E94F12E2EE333ECB9
:102730004EE259E30E94013020E030E040EC5EE3DD
:102740000E94EE2D60937202709373028093740264
:102750009093750289C010927703109278031092BB
:10276000790310927A03CE0183709927892BE1F0C7
:10277000BE016170772780E090E00E94EF2E20E09C
:1027800030E040E05EE30E94013020E030E040E4D1
:102790005FE30E94EE2D6093720270937302809348
:1027A0007402909375020CC080E090E0A0E0BFE35B
:1027B0008093720290937302A0937402B093750297
:1027C000C770DD27CD2B09F04FC010927202109216
:1027D0007302109274021092750246C01092770331
:1027E000109278031092790310927A0300E010E0BF
:1027F00020E03FE30093720210937302209374026F
:10280000309375026739710578F180E090E00E949D
:10281000EF2E20E030E047E153E40E94ED2D20E070
:1028200030E04AE754E40E94562E20E030E048E4CD
:1028300052E40E94013020E030E040EA51E40E947E
:10284000332F0E94BE2E660F771F660F771FFB0186
:10285000EC50FD4F2081318142815381C701B60187
:102860000E9401306B017C01C701B601DF91CF915D
:102870001F910F91FF90EF90DF90CF90BF90AF909E
:102880009F908F9008958091D8030895CF93DF9300
:1028900000D01F92CDB7DEB79C0180915E048430DA
:1028A00019F593E099833B832A839093E9008FEF96
:1028B0009091E800815095FD06C095ED9A95F1F74D
:1028C00000008111F5CF8091E80085FF0DC040E048
:1028D00050E063E070E0CE0101960E94A71680915F
:1028E000E8008E778093E8000F900F900F90DF91B3
:1028F000CF910895CF93DF9300D01F92CDB7DEB76D
:1029000020915E04243021F522E029839B838A8371
:1029100083E08093E9008FEF9091E800815095FD6E
:1029200006C095ED9A95F1F700008111F5CF8091E1
:10293000E80085FF0DC040E050E063E070E0CE01AC
:1029400001960E94A7168091E8008E778093E80098
:102950000F900F900F90DF91CF91089520915E041A
:102960002430F1F422E02093E9002FEF3091E800C9
:10297000215035FD06C035ED3A95F1F700002111E3
:10298000F5CF2091E80025FF0BC040E050E065E066
:1029900070E00E94A7168091E8008E778093E8008F
:1029A0000895CF93DF93EC0190915E04943009F089
:1029B00046C0809184028823D9F0809185028823C3
:1029C000B9F09093E9008FEF9091E800815095FD68
:1029D00006C095E19A95F1F700008111F5CF80913D
:1029E000E80085FF2CC040E050E060E170E017C0D7
:1029F00081E08093E9008FEF9091E800815095FD90
:102A000006C095ED9A95F1F700008111F5CF809100
:102A1000E80085FF14C040E050E068E070E0CE01BF
:102A20000E94A7168091E8008E778093E80080E1ED
:102A3000FE01A8ECB3E001900D928A95E1F7DF91D9
:102A4000CF91089580915D04811109C00E943C18C6
:102A50000E9499188091E20084608093E2000895BA
:102A600010925D040895089508950C94E12742E0C2
:102A700061EC81E00E94B61742E061EC82E00E94C6
:102A8000B61742E061EC83E00E94B61742E161ECC8
:102A900084E00C94B61780916004833009F455C02B
:102AA00030F4813071F0823009F48EC008958A309C
:102AB00009F47AC08B3009F460C0893009F09CC0F9
:102AC00020C080915F04813A09F096C08091E800AF
:102AD000877F8093E8008091630490916404892B40
:102AE00021F460E188EC93E003C060E080E090E0D6
:102AF00070E00E94F2168091E8008B778093E800E6
:102B0000089580915F04813209F076C0809163045A
:102B100090916404009719F0039709F06DC08091BB
:102B2000E800877F8093E8008091E80082FD05C07F
:102B300080915E048111F8CF5FC08091F100809395
:102B4000D8038091E8008B7753C080915F04813A6D
:102B500009F052C08091630490916404892B09F0BC
:102B60004BC08091E800877F8093E8008091E80067
:102B700080FFFCCF8091840236C080915F04813257
:102B8000D9F58091630490916404892BA9F5809113
:102B9000E800877F8093E8000E94EB178091610432
:102BA000809384020C945C2180915F04813221F532
:102BB0008091E800877F8093E8000E94EB17809166
:102BC00062048093D903089580915F04813AA1F44F
:102BD0008091E800877F8093E8008091E80080FF83
:102BE000FCCF8091D9038093F1008091E8008E772B
:102BF0008093E8000C94EB17089584B7877F84BF17
:102C000088E10FB6F89480936000109260000FBEC8
:102C100090E080E80FB6F894809361009093610093
:102C20000FBE0E948E1B0E943C180E949918809132
:102C3000E20084608093E20078940E941F1B0E944F
:102C4000901B8AE792E00E943A1B80915E048530D7
:102C500069F40E949B2780915C048823B1F30E9451
:102C6000C927882391F30E949116EFCF0E94981BE9
:102C7000ECCF292F332723303105C9F064F42130FC
:102C8000310581F02230310509F043C08DE690E036
:102C90002AE338E042C021323105F1F02232310519
:102CA00041F137C082E190E027EA38E036C0992749
:102CB0008130910541F08230910541F0892B49F531
:102CC000E6E3F8E005C0E8E0F8E002C0EEEDF7E08A
:102CD000849190E09F0121C06430D8F4E62FF0E0A9
:102CE000EE0FFF1FE05BFC4F2081318189E090E017
:102CF00014C0643070F470E0FB01EE0FFF1FE85B5E
:102D0000FC4F20813181FB01EC5BFC4F808190E026
:102D100004C080E090E020E030E0FA0131832083BD
:102D2000089580E189BD82E189BD09B400FEFDCF2F
:102D30008091D8008F7D8093D8008091E0008260E0
:102D40008093E0008091E00081FDFCCF0895CF9258
:102D5000DF92EF92FF920F931F93CF93DF93EC01DB
:102D60008B016A010E940A18811133C0C114D10479
:102D700039F0F60180819181081B190BC80FD91F0A
:102D8000E12CF12C0115110519F18091E80085FD68
:102D900016C08091E8008E778093E800C114D104BA
:102DA00049F0F60180819181E80EF91EF182E082FE
:102DB00085E00FC00E940A18882321F30AC0899178
:102DC0008093F10001501109FFEFEF1AFF0ADACFEB
:102DD00080E0DF91CF911F910F91FF90EF90DF90F6
:102DE000CF90089520916504309166042617370727
:102DF00048F06115710539F42091E8002E77209391
:102E0000E80001C0B90140E061157105A9F1209108
:102E10005E04222309F443C0253009F442C0209106
:102E2000E80023FD40C02091E80022FD32C020913F
:102E3000E80020FFE9CF4091F3002091F20030E05C
:102E4000342BFC01CF016115710559F02830310593
:102E500040F481918093F100615071092F5F3F4FE1
:102E6000F1CF41E02830310509F040E02091E80041
:102E70002E772093E800C8CF4111C9CF0AC08091B6
:102E80005E04882361F0853061F08091E80083FD65
:102E90000AC08091E80082FFF2CF80E0089582E0CE
:102EA000089583E0089581E00895209165043091AC
:102EB00066042617370748F06115710539F420912B
:102EC000E8002E772093E80001C0B901FC0120E062
:102ED0006115710591F180915E04882309F440C069
:102EE000853009F43FC08091E80083FD3DC08091AA
:102EF000E80082FD2FC08091E80080FFE9CF20919B
:102F0000F3008091F20090E0922B6115710559F069
:102F10008830910540F424912093F100319661505E
:102F200071090196F2CF21E0089709F020E0809125
:102F3000E8008E778093E800CBCF2111CCCF0AC078
:102F400080915E04882361F0853061F08091E80013
:102F500083FD0AC08091E80082FFF2CF80E00895EF
:102F600082E0089583E0089581E00895982F9730D6
:102F700058F59093E900981739F07091EC00209182
:102F8000ED005091F00003C0242F762F50E021FF78
:102F900019C03091EB003E7F3093EB003091ED0093
:102FA0003D7F3093ED003091EB0031603093EB00CA
:102FB0007093EC002093ED005093F0002091EE0010
:102FC00027FF07C09F5FD3CF8F708093E90081E018
:102FD000089580E0089580915F0487FF11C080917B
:102FE000E80082FD05C080915E048111F8CF11C018
:102FF0008091E8008B770BC080915E04882349F0B4
:103000008091E80080FFF8CF8091E8008E77809370
:10301000E80008952091E4003091E50095E64091A4
:10302000EC00842F817040FF22C08091E80080FD79
:103030001CC080915E04882391F0853091F08091CE
:10304000EB0085FD10C04091E4005091E50042176F
:10305000530729F39A01915011F784E0089582E013
:10306000089583E0089581E0089580E008954091F7
:10307000E80042FFDECF08950E94AA180E94B2180D
:10308000E0EEF0E0808181608083E8EDF0E0808117
:103090008F77808319BCA7EDB0E08C918E7F8C93E5
:1030A00080818F7E808310925D0408950F931F931B
:1030B000CF93DF930E94AA180E94B218C8EDD0E007
:1030C00088818F77888388818068888388818F7DD5
:1030D000888319BC10925E0410925A0410925C040A
:1030E00010925B0400EE10E0F80180818B7F8083FA
:1030F00088818160888342E060E080E00E94B617AA
:10310000E1EEF0E080818E7F8083E2EEF0E080816E
:1031100081608083808188608083F80180818E7FD8
:103120008083888180618883DF91CF911F910F9187
:103130000895E8EDF0E080818F7E8083E7EDF0E098
:1031400080818160808384E082BF81E080935D0420
:103150000C945618E8EDF0E080818E7F8083109209
:10316000E20008951092DA001092E10008951F9293
:103170000F920FB60F9211242F933F934F935F93AB
:103180006F937F938F939F93AF93BF93EF93FF932F
:103190008091E10082FF0BC08091E20082FF07C0B6
:1031A0008091E1008B7F8093E1000E941E1B809143
:1031B000DA0080FF1FC08091D80080FF1BC0809183
:1031C000DA008E7F8093DA008091D90080FF0DC0F5
:1031D00080E189BD82E189BD09B400FEFDCF81E0B7
:1031E00080935E040E94221505C019BC10925E04F3
:1031F0000E9430158091E10080FF19C08091E200AB
:1032000080FF15C08091E2008E7F8093E200809164
:10321000E20080618093E2008091D8008062809318
:10322000D80019BC85E080935E040E94341580911B
:10323000E10084FF30C08091E20084FF2CC080E177
:1032400089BD82E189BD09B400FEFDCF8091D8001F
:103250008F7D8093D8008091E1008F7E8093E10084
:103260008091E2008F7E8093E2008091E200816095
:103270008093E20080915A04882311F084E007C013
:103280008091E30087FD02C081E001C083E080936C
:103290005E040E9435158091E10083FF29C0809172
:1032A000E20083FF25C08091E100877F8093E100E9
:1032B00082E080935E0410925A048091E1008E7F38
:1032C0008093E1008091E2008E7F8093E200809104
:1032D000E20080618093E20042E060E080E00E94D2
:1032E000B6178091F00088608093F0000E9433153B
:1032F000FF91EF91BF91AF919F918F917F916F91CE
:103300005F914F913F912F910F900FBE0F901F90A3
:1033100018951F920F920FB60F9211242F933F937F
:103320004F935F936F937F938F939F93AF93BF93CD
:10333000CF93DF93EF93FF93C091E900CF7080911B
:10334000EC00D82FD17080FDD0E81092E900809178
:10335000F000877F8093F00078940E94CD1910923E
:10336000E9008091F00088608093F000CD2BCF7051
:10337000C093E900FF91EF91DF91CF91BF91AF91A1
:103380009F918F917F916F915F914F913F912F917D
:103390000F900FBE0F901F9018951F93CF93DF9340
:1033A000CDB7DEB7AA970FB6F894DEBF0FBECDBF7C
:1033B000EFE5F4E088E08E0F9091F10091938E1389
:1033C000FBCF0E944B158091E80083FF1FC18091C5
:1033D0005F0490916004492F50E04A30510508F095
:1033E00015C1FA01EC59FF4F0C94E331803881F09C
:1033F000823809F00BC1809163048F708093E900DB
:103400008091EB0085FB882780F91092E90006C0C7
:1034100080915B0490915C04911182609091E8002E
:10342000977F9093E8008093F1001092F100C8C05C
:10343000282F2D7F09F0EAC0882319F0823061F02F
:10344000E5C080916104813009F0E0C0933009F05B
:1034500080E080935C042BC080916104811127C0BF
:10346000809163048F7009F4D1C08093E9002091AA
:10347000EB0020FF1CC0933021F48091EB008062B0
:1034800014C09091EB0090619093EB0021E030E04C
:10349000A90102C0440F551F8A95E2F74093EA0044
:1034A0001092EA008091EB0088608093EB0010920C
:1034B000E9008091E800877F86C08111A7C0109144
:1034C00061041F778091E3008078812B8093E30073
:1034D0008091E800877F8093E8000E94EB1780913D
:1034E000E80080FFFCCF8091E30080688093E300D8
:1034F000111102C082E001C083E080935E0486C0A7
:103500008058823008F082C08091610490916204FA
:103510008C3D53E0950779F583E08A838AE28983BD
:103520004FB7F894DE01139620E03EE051E2E32F1E
:10353000F0E050935700E49120FF03C0E295EF7054
:103540003F5FEF708E2F90E0EA3010F0C79601C019
:10355000C0968D939D932F5F243149F74FBF809183
:10356000E800877F8093E8006AE270E0CE01019670
:103570000E94F21614C0AE014F5F5F4F609163046A
:103580000E943916BC01009709F440C09091E800F0
:10359000977F9093E80089819A810E9455178091C6
:1035A000E8008B778093E80031C0803879F580910E
:1035B000E800877F8093E80080915A048093F100AF
:1035C0008091E8008E778093E8000E94EB171EC080
:1035D00081111CC0909161049230C0F48091E80088
:1035E000877F8093E80090935A040E94EB178091A4
:1035F0005A04811106C08091E30087FD02C081E07A
:1036000001C084E080935E040E9437158091E80039
:1036100083FF0AC08091E800877F8093E800809153
:10362000EB0080628093EB00AA960FB6F894DEBFA1
:103630000FBECDBFDF91CF911F9108950895CF9315
:1036400080915E048823A1F0C091E900CF70909131
:10365000EC00892F817090FD80E8C82B1092E90062
:103660008091E80083FD0E94CD19CF70C093E900DE
:10367000CF9108959093DF038093DE030895E09146
:10368000DE03F091DF03309721F00190F081E02D0F
:10369000099480E00895E091DE03F091DF03309714
:1036A00021F00280F381E02D09940895E091DE037A
:1036B000F091DF03309721F00480F581E02D09942B
:1036C00008952091DC033091DD038217930771F098
:1036D0009093DD038093DC03E091DE03F091DF0340
:1036E000309721F00680F781E02D0994089520910C
:1036F000DA033091DB038217930771F09093DB03B9
:103700008093DA03E091DE03F091DF03309721F03C
:103710000084F185E02D0994089508950C948D1B83
:103720000E9415280E94760B0E949B280C94562D0F
:103730004F925F927F928F929F92AF92BF92CF9261
:10374000DF92EF92FF920F931F93CF93DF93CDB74A
:10375000DEB72A970FB6F894DEBF0FBECDBF0E942A
:10376000650C91EEC92E93E0D92E00E010E0AA245A
:10377000A394B12C702E802F0E94AE0D4C01F60147
:10378000419051906F014826592641145104B1F4DB
:103790000F5F1F4F0430110569F78FEF89838A830C
:1037A0001B820E941E288160782F9D838C83498113
:1037B0005A816B818D810E94511C3AC080913D04D9
:1037C00081FD0E94B70D20E030E07501022E02C09D
:1037D000EE0CFF1C0A94E2F7C70184219521892B86
:1037E00009F12E837F828E209F2091E0892809F4A1
:1037F00090E098870E941E288160782F9A87898799
:103800004E815F8168858A850E94511C000F111FBF
:10381000F801EF51FC4F80819181E826F926F18271
:10382000E08206C02F5F3F4F2C30310571F6B0CFDC
:103830000E94872A1091E0030E943F1B1817D9F0BD
:103840000E943F1B8093E0032A960FB6F894DEBFD8
:103850000FBECDBFDF91CF911F910F91FF90EF90E1
:10386000DF90CF90BF90AF909F908F907F905F90B0
:103870004F900C94AE0A2A960FB6F894DEBF0FBE96
:10388000CDBFDF91CF911F910F91FF90EF90DF900F
:10389000CF90BF90AF909F908F907F905F904F9010
:1038A0000895CF93DF93CDB7DEB72B970FB6F8947B
:1038B000DEBF0FBECDBF4F83588769877A878B875E
:1038C000DE01119686E0FD0111928A95E9F785E007
:1038D000FE01379601900D928A95E1F749815A8150
:1038E0006B817C818D819E810E94F6232B960FB681
:1038F000F894DEBF0FBECDBFDF91CF910895CF9377
:10390000882309F4C2C0C82F823859F40E943F1B93
:1039100081FDBBC089E30E949F260E946C2789E33A
:103920000CC0833879F40E943F1B80FDAEC083E554
:103930000E949F260E946C2783E50E94E126CF917A
:103940000C946C27843859F40E943F1B82FD9DC063
:1039500087E40E949F260E946C2787E4EECF8CEFBD
:103960008C0F813A48F48C2F0E94BE2C81118DC09F
:103970008C2F0E949F26E3CF80E28C0F883048F482
:10398000C77081E001C0880FCA95EAF70E94252719
:10399000D6CF8BE58C0F833078F4C53A29F0C63A40
:1039A00031F083E890E005C081E890E002C082E851
:1039B00090E0CF910C94611B88E58C0F833108F067
:1039C00064C0C83A39F1C93A41F1CA3A49F1CB3A2F
:1039D00051F1CC3A59F1CD3A61F1C03B69F1CE3A9F
:1039E00071F1CF3A79F1C13B81F1C23B89F1C33B1F
:1039F00091F1C43B99F1C53BA1F1C63BA9F1C73B8D
:103A0000B1F1C83BB9F1C93BC1F1CA3BC9F180E092
:103A100090E038C082EE90E035C089EE90E032C090
:103A20008AEE90E02FC085EB90E02CC086EB90E012
:103A300029C087EB90E026C08CEC90E023C08DEC91
:103A400090E020C083E891E01DC08AE891E01AC0B0
:103A500082E991E017C084E991E014C081E292E02C
:103A600011C083E292E00EC084E292E00BC085E2D6
:103A700092E008C086E292E005C087E292E002C0D0
:103A80008AE292E0CF910C94771BCF91089588231E
:103A900009F44BC0823859F40E943F1B81FF45C096
:103AA00089E30E949F260E946C2789E30CC083381B
:103AB00071F40E943F1B80FF38C083E50E949F265F
:103AC0000E946C2783E50E94E1260C946C278438C1
:103AD00059F40E943F1B82FF28C087E40E949F2662
:103AE0000E946C2787E4EFCF9CEF980F913A58F330
:103AF00090E2980F983050F4877091E001C0990FD0
:103B00008A95EAF7892F0E942B27DFCF9BE5980F34
:103B1000933020F480E090E00C94611B885A83314C
:103B200020F480E090E00C94771B0895882321F026
:103B30000E9425270C946C270895882321F00E9469
:103B40002B270C946C270895BF92CF92DF92EF92AF
:103B5000FF920F931F93CF93DF9300D000D000D03C
:103B6000CDB7DEB725E0FC01DE01119601900D9284
:103B70002A95E1F7FC01D0801181028125812295EF
:103B80002F7043815481452B09F472C31F3F21F4E8
:103B9000FFEFDF1609F46CC37C012E830E947707C8
:103BA000D9821A8369817A81802F0E949B26182FDF
:103BB000B92E0E9450260E9417252E81002319F04D
:103BC0000E9442272E81EB2DE295EF70F0E0E25942
:103BD000FF4F0C94E3318B2D807F9B2D9F70F92E2E
:103BE000882319F0F29480EFF822002389F0FF2057
:103BF00009F47CC280E2810F883020F48F2D0E946E
:103C0000252703C08F2D0E9435270E946C276EC286
:103C1000812F0E94471DFF2009F42AC3105E8F2DBB
:103C2000183018F40E942B2702C00E943B272696CA
:103C30000FB6F894DEBF0FBECDBFDF91CF911F91BD
:103C40000F91FF90EF90DF90CF90BF900C946C2776
:103C50008B2D807F9B2D9F70803211F4892F03C0A4
:103C6000892F8295807F112319F0113011F12BC01B
:103C70000023A9F0222389F1213079F526960FB689
:103C8000F894DEBF0FBECDBFDF91CF911F910F9192
:103C9000FF90EF90DF90CF90BF900C945527222398
:103CA00019F0213009F4E4C28E830E9458278E81D6
:103CB0009BC1002321F0263008F0DAC20EC0253067
:103CC00008F0D6C291C10023C9F0222331F0F701D8
:103CD000958190FF0BC29F70958326960FB6F8943E
:103CE000DEBF0FBECDBFDF91CF911F910F91FF902F
:103CF000EF90DF90CF90BF900C94961D222309F493
:103D000073C109C22B2D26952695237030E021150D
:103D1000310521F021303105D1F0AAC2002321F074
:103D2000812F9B2D937002C080E090E026960FB605
:103D3000F894DEBF0FBECDBFDF91CF911F910F91E1
:103D4000FF90EF90DF90CF90BF900C94611B002309
:103D500021F0812F9B2D937002C080E090E0269689
:103D60000FB6F894DEBF0FBECDBFDF91CF911F918C
:103D70000F91FF90EF90DF90CF90BF900C94771B46
:103D8000812F002319F00E948F2902C00E94F72979
:103D900026960FB6F894DEBF0FBECDBFDF91CF9150
:103DA0001F910F91FF90EF90DF90CF90BF900C94F8
:103DB0007C2A8B2D837009F07BC0011159C2812FA1
:103DC000829586958770880F880F912F9F70C92ED6
:103DD000D12CE12CF12C082E04C0CC0CDD1CEE1CE7
:103DE000FF1C0A94D2F714FF12C04FE050E060E0CD
:103DF00070E004C0440F551F661F771F8A95D2F7E5
:103E0000CB01BA01609570958095909503C060E0F4
:103E100070E0CB012B2D269526952370422F50E084
:103E200042305105D9F04330510569F16C297D29A3
:103E30008E299F294130510551F126960FB6F894ED
:103E4000DEBF0FBECDBFDF91CF911F910F91FF90CD
:103E5000EF90DF90CF90BF900C943E256C297D2988
:103E60008E299F2926960FB6F894DEBF0FBECDBFD0
:103E7000DF91CF911F910F91FF90EF90DF90CF9046
:103E8000BF900C945A250E943E25C701B601269684
:103E90000FB6F894DEBF0FBECDBFDF91CF911F915B
:103EA0000F91FF90EF90DF90CF90BF900C94222560
:103EB000002319F08B2D817001C08695882309F4A9
:103EC000D7C1812F829586958770880F880F912F93
:103ED0009F70C92ED12CE12CF12C082E04C0CC0CE3
:103EE000DD1CEE1CFF1C0A94D2F714FF12C04FE039
:103EF00050E060E070E004C0440F551F661F771F5C
:103F00008A95D2F7CB01BA0160957095809590950E
:103F100003C060E070E0CB012B2D26952695237021
:103F2000422F50E042305105D9F04330510569F13C
:103F30006C297D298E299F294130510551F1269602
:103F40000FB6F894DEBF0FBECDBFDF91CF911F91AA
:103F50000F91FF90EF90DF90CF90BF900C941826B8
:103F60006C297D298E299F2926960FB6F894DEBFED
:103F70000FBECDBFDF91CF911F910F91FF90EF90BA
:103F8000DF90CF90BF900C9434260E941826C70172
:103F9000B60126960FB6F894DEBF0FBECDBFDF91F7
:103FA000CF911F910F91FF90EF90DF90CF90BF9036
:103FB0000C94FC25103F49F118F4103E48F491C0D0
:103FC000123F09F453C0E8F1133F09F464C089C0FB
:103FD0001F708B2D8F71002321F00E949525812F5A
:103FE0007CCE0E94B625812F26960FB6F894DEBFB0
:103FF0000FBECDBFDF91CF911F910F91FF90EF903A
:10400000DF90CF90BF900C949D1D0023B1F0253020
:1040100008F02EC18B2D8F7126960FB6F894DEBF57
:104020000FBECDBFDF91CF911F910F91FF90EF9009
:10403000DF90CF90BF900C94DB25263008F018C19C
:10404000E9CF0023A9F08B2D8F7126960FB6F89437
:10405000DEBF0FBECDBFDF91CF911F910F91FF90BB
:10406000EF90DF90CF90BF900C949525002359F3EB
:104070008B2D8F7126960FB6F894DEBF0FBECDBF85
:10408000DF91CF911F910F91FF90EF90DF90CF9034
:10409000BF900C94B625002399F08B2D8F71269636
:1040A0000FB6F894DEBF0FBECDBFDF91CF911F9149
:1040B0000F91FF90EF90DF90CF90BF900C948025F0
:1040C00026960FB6F894DEBF0FBECDBFDF91CF911D
:1040D0001F910F91FF90EF90DF90CF90BF900C94C5
:1040E00076250023A9F0222309F4ADCF812F26964F
:1040F0000FB6F894DEBF0FBECDBFDF91CF911F91F9
:104100000F91FF90EF90DF90CF90BF900C947F1CA9
:10411000222309F4ADCF812F26960FB6F894DEBF87
:104120000FBECDBFDF91CF911F910F91FF90EF9008
:10413000DF90CF90BF900C94471D4B2D4F70612F97
:10414000C7010E94690526960FB6F894DEBF0FBE20
:10415000CDBFDF91CF911F910F91FF90EF90DF9036
:10416000CF90BF900C949A24011182C09B2D9F7018
:10417000492F50E04230510509F443C0C4F44115C1
:10418000510571F14130510509F072C026960FB604
:10419000F894DEBF0FBECDBFDF91CF911F910F917D
:1041A000FF90EF90DF90CF90BF900C947E2D433026
:1041B0005105C1F14430510509F05AC0812F2696AE
:1041C0000FB6F894DEBF0FBECDBFDF91CF911F9128
:1041D0000F91FF90EF90DF90CF90BF900C94D02D77
:1041E00026960FB6F894DEBF0FBECDBFDF91CF91FC
:1041F0001F910F91FF90EF90DF90CF90BF900C94A4
:10420000672D26960FB6F894DEBF0FBECDBFDF91A7
:10421000CF911F910F91FF90EF90DF90CF90BF90C3
:104220000C949A2D26960FB6F894DEBF0FBECDBF24
:10423000DF91CF911F910F91FF90EF90DF90CF9082
:10424000BF900C94AD2D4B2D4F70612FC70126965A
:104250000FB6F894DEBF0FBECDBFDF91CF911F9197
:104260000F91FF90EF90DF90CF90BF900C94790763
:1042700026960FB6F894DEBF0FBECDBFDF91CF916B
:104280001F910F91FF90EF90DF90CF90BF90089516
:104290000E9442270E9452270E9417270E946C27E3
:1042A0000E942D2B0E947C2A80E090E00E94611BDE
:1042B00080E090E00C94771B0E9432270C944821F8
:1042C0000E949026292F22952F7030E02C30310546
:1042D0004CF42A3031056CF422503109223031057A
:1042E00088F407C02C30310549F02F30310531F00A
:1042F00009C0803E48F0803F29F406C093FB882720
:1043000080F9089580E0089581E00895CF93DF93C8
:1043100000D000D01F92CDB7DEB70F900F900F9056
:104320000F900F90DF91CF910895CF93DF9300D03E
:1043300000D000D0CDB7DEB726960FB6F894DEBF1A
:104340000FBECDBFDF91CF9108951F93CF93DF9321
:10435000C091E90316E08091EA03C81799F0D0E014
:104360001C9FF0011D9FF00D1124E551FC4F408171
:10437000518162817381848195810E94952121966A
:10438000C770E9CFDF91CF911F91089540911B0431
:1043900050911C0460911D0470911E0480911F04B3
:1043A000909120040C9495218091200482958F7027
:1043B00009F054C080911D04882309F44FC08091F6
:1043C000E903A091EA0360911B0470911C044091E1
:1043D0001E0450911F04B6E08A1709F43FC090E014
:1043E00041155105C1F17F3F11F46F3FA1F1B89F15
:1043F000F001B99FF00D1124E551FC4F218172139A
:104400002AC02081621327C02281211124C0238168
:1044100034812417350710F421503109241B350B42
:10442000283C3105C0F4209120042F702061209396
:10443000200426E0289FF001299FF00D1124E0516F
:10444000FC4F80818F70806180838BE194E00E94BB
:10445000A41D0C94A52101968770BECF0895CF921C
:10446000DF92EF92FF920F931F93CF93DF93CDB71D
:10447000DEB762970FB6F894DEBF0FBECDBF8C01DA
:1044800085E0F801DE011D9601900D928A95E1F715
:10449000D8014C9111965C91119712966C911297DC
:1044A0001396CD90DC90149730911B0470911C04EE
:1044B00080911E0490911F04009709F46BC17F3F07
:1044C00019F43F3F09F466C1E0901D04EE2009F4A1
:1044D000C0C020912004C816D90628F0F601E81BB8
:1044E000F90BCF0104C0809590958C0D9D1DFF2484
:1044F000F394883C910578F0F12C207F09F0C6C038
:104500007C2DD98AC88A89890E9486218BE194E012
:104510000E94A41DB1C0822F807F09F046C0751390
:1045200014C0341312C0611110C02F702061209389
:1045300020040E94C6218BE194E00E94A41D80917A
:104540002004D80115968C932EC0CD2819F15F3F19
:1045500011F44F3FF9F0F62E61111CC08091E90370
:104560002091EA0336E0821709F45AC090E0389FA0
:10457000F001399FF00D1124E551FC4F7181571363
:1045800006C07081471303C07281711103C0019688
:104590008770E9CFF62E662309F418C180912004B4
:1045A000816080932004F12C11C1751308C034136D
:1045B00006C0611104C080912004D801C3C04D879A
:1045C0005E878D859E856A8B0E9460216A8988231B
:1045D000E1F16623D1F120912004822F82958F7022
:1045E00090E0029774F080911B0490911C049887CE
:1045F0008F831986DB86CA862C87CE0107960E9498
:10460000A41D86E0F801ABE1B4E001900D928A951B
:10461000E1F70E94D4210E94C621FF24F394D6C062
:104620004D875E878D859E850E949026292F229535
:104630002F7030E0223031050CF0BCC09F7009F0C3
:10464000B6C0805E883008F4C1C0C8010E94A41DB5
:10465000E4CFC816D90608F453C0F601E81BF90BDD
:10466000CF01883C910508F450C0F12C7C2DD98AEB
:10467000C88A89890E948621EBE1F4E086E0DF01A7
:104680001D928A95E9F70E94C621A0C0751314C037
:10469000341312C0611110C080912004F801858389
:1046A000C8010E94A41D86E0EBE1F4E0DF011D9249
:1046B0008A95E9F7FE2C8AC04D875E878D859E8599
:1046C0006A8B0E9460216A89882309F4BECF662321
:1046D00009F4BBCF20912004822F82958F7090E047
:1046E00002970CF48ECF80911B0490911C049A8346
:1046F00089831B82DD82CC822E83CE0101967FCFFF
:10470000809590958C0D9D1DACCFF62E662309F4F7
:104710009CCF75132EC034132CC02091200420FD93
:104720001FC0822F82958F70D9F0D80115962C93D7
:1047300015978F3049F08F5F982F9295907F822F39
:104740008F70892B15968C93C8010E94A41D86E05A
:10475000F801ABE1B4E001900D928A95E1F793CFB7
:1047600086E0F801ABE1B4E001900D928A95E1F7A3
:104770002DC04D875E878D859E850E9460218111A9
:1047800040CF80912004816080932004C8010E9462
:10479000A41D1CC0662309F458CF4D875E878D8504
:1047A0009E850E946021882309F44FCF2ACF811172
:1047B00048CF0CC0243031050CF047CF9F7009F46E
:1047C00040CFF8019581907F09F03BCF8F2D629605
:1047D0000FB6F894DEBF0FBECDBFDF91CF911F9112
:1047E0000F91FF90EF90DF90CF9008951F93CF939C
:1047F000DF93CDB7DEB72C970FB6F894DEBF0FBEB0
:10480000CDBF4F83588769877A878B879C87CE0176
:1048100007960E942F22882369F08F8198852A8528
:104820003B85232BF1F19F3F09F063C08F3F09F0D7
:1048300060C037C086E0FE013796DE011196019018
:104840000D928A95E1F76F817885EA85FB8530972F
:1048500041F17F3F11F46F3F21F12091EA0330E0F5
:10486000C9010196877099274091E90350E08417A8
:10487000950709F447C069837A83FD83EC8396E04A
:10488000929FD001939FB00D1124A551BC4FFE0102
:10489000319601900D929A95E1F78093EA030E9478
:1048A000A52116E08091E9039091EA038917C1F1EF
:1048B000189FC001112485519C4F0E942F228823EC
:1048C00079F1E091E9031E9FF0011124E551FC4FBD
:1048D0004081518162817381848195810E949521FB
:1048E0008091E90390E00196877099278093E9030E
:1048F000D9CF4F81588569857A858B859C850E94A3
:104900009521CFCF0E945C211092EA031092E90317
:10491000EBE1F4E086E0DF011D928A95E9F7C1CF73
:104920002C960FB6F894DEBF0FBECDBFDF91CF91AE
:104930001F910895EF92FF920F931F93CF93DF93F0
:104940008C01009709F46CC0F12CEE24E394E8018B
:104950002196F8018491843740F4843008F051C0E6
:10496000813081F0823019F15BC0853709F444C091
:10497000A8F19CE7980F903708F052C08F770E94FB
:10498000471D41C00E5F1F4FFE01C49180E28C0F96
:10499000883048F4C7708E2D01C0880FCA95EAF799
:1049A0000E94452714C08C2F0E947F1C2DC00E5FD3
:1049B0001F4FFE01C49180E28C0F883058F4C770FD
:1049C0008E2D01C0880FCA95EAF70E944B270E94DE
:1049D0006C271AC08C2F0E94471D16C00E5F1F4FF8
:1049E000FE01C491CC2381F08FE99FE00197F1F79C
:1049F00000C00000C150F6CF0E5F1F4FFE01F490C3
:104A000003C00E947F1C8E018F2D882309F49FCF45
:104A1000EFE9FFE03197F1F700C000008150F5CFDA
:104A2000DF91CF911F910F91FF90EF90089508951E
:104A300060932504709326048093270490932804A0
:104A40000C9448210F931F93009125041091260484
:104A50002091270430912804DC01CB01802B912B7D
:104A6000A22BB32B8093250490932604A0932704B4
:104A7000B09328041F910F910C9448210F931F931A
:104A800000912504109126042091270430912804D8
:104A9000DC01CB0180239123A223B323809325043F
:104AA00090932604A0932704B09328041F910F919C
:104AB0000C9448210F931F93009125041091260414
:104AC0002091270430912804DC01CB018027912715
:104AD000A227B3278093250490932604A09327044C
:104AE000B09328041F910F910C9448211092210437
:104AF0001092220410922304109224040C94482152
:104B000041E050E060E070E004C0440F551F661FB4
:104B1000771F8A95D2F74093210450932204609323
:104B20002304709324040C94482141E050E060E099
:104B300070E004C0440F551F661F771F8A95D2F797
:104B40008091210490912204A0912304B091240427
:104B5000482B592B6A2B7B2B409321045093220422
:104B600060932304709324040C94482141E050E0A6
:104B700060E070E004C0440F551F661F771F8A95E0
:104B8000D2F7409550956095709580912104909151
:104B90002204A0912304B0912404482359236A23BA
:104BA0007B23409321045093220460932304709349
:104BB00024040C94482141E050E060E070E004C01F
:104BC000440F551F661F771F8A95D2F780912104E5
:104BD00090912204A0912304B091240448275927DE
:104BE0006A277B2740932104509322046093230477
:104BF000709324040C9448210F931F930091210477
:104C0000109122042091230430912404DC01CB0173
:104C1000802B912BA22BB32B809321049093220401
:104C2000A0932304B09324041F910F910C94482166
:104C30000F931F93009121041091220420912304CB
:104C400030912404DC01CB0180239123A223B323E0
:104C50008093210490932204A0932304B09324040E
:104C60001F910F910C9448210F931F9300912104E1
:104C7000109122042091230430912404DC01CB0103
:104C800080279127A227B3278093210490932204A1
:104C9000A0932304B09324041F910F910C944821F6
:104CA0000895CF92DF92EF92FF920F931F93CF93CD
:104CB000DF938C01C0902504D0902604E090270457
:104CC000F09028048091210490912204A091230463
:104CD000B0912404C82AD92AEA2AFB2ACFE1D0E0DD
:104CE000D701C6010C2E04C0B695A7959795879558
:104CF0000A94D2F780FF06C0B8018C2F0E94D30916
:104D0000019721F4219760F780E001C08C2FDF919B
:104D1000CF911F910F91FF90EF90DF90CF9008956A
:104D2000CF93DF93EC010E945126BE010E94D3096C
:104D3000DF91CF910895CB010E9490260895909124
:104D40008402992321F090918502911109C020914C
:104D5000860230918702F90132969FEF40E01FC032
:104D6000982F9695969596959F3050F5E0918602EE
:104D7000F0918702E90FF11D877021E030E0A90171
:104D800002C0440F551F8A95E2F7CA019181892B11
:104D9000818308959F3F39F04F5F4E3041F051912C
:104DA0005813F8CF0DC05111F7CF942FF5CF9F3F77
:104DB00039F0F901E90FF11D97FDFA958283089505
:104DC000089590918402992321F090918502911188
:104DD00009C02091860230918702F9013296205F46
:104DE0003F4F1FC0982F9695969596959F30F0F45B
:104DF000E0918602F0918702E90FF11D877021E0B2
:104E000030E0A90102C0440F551F8A95E2F7CA019C
:104E1000809591818923818308953196E217F30764
:104E200029F090819813F9CF1082F7CF089581E08F
:104E300090E0E0918602F0918702E80FF91F10825E
:104E4000019680319105A9F7089590913C04892B32
:104E500080933C040895809590913C04892380932D
:104E60003C04089510923C04089590913B04892BD2
:104E700080933B040895809590913B04892380930F
:104E80003B04089510923B04089590913A04892BB5
:104E900080933A040895809590913A0489238093F1
:104EA0003A04089510923A040895809329040895CD
:104EB0001092290408958091860290918702FC0146
:104EC00031969C01205F3F4F80E0919191118F5F5F
:104ED000E217F307D1F70895E0918602F091870277
:104EE00080913C048083E0918602F091870290815A
:104EF00080913B04892B8083E0918602F0918702A8
:104F0000908180913A04892B8083809129048823A1
:104F100061F0E0918602F09187029081892B808375
:104F20000E945B2781111092290480918602909142
:104F300087020C944B1B80915E04843039F11092EF
:104F40003E0420E488E190E00FB6F894A8958093A1
:104F500060000FBE2093600080E00E94300580E07A
:104F60000E94AE0A83B7817F846083BF83B781606C
:104F700083BF7894889583B78E7F83BF88E10FB60F
:104F8000F89480936000109260000FBE0895089519
:104F90000895CF9380E00E9430050E94C7270E94A9
:104FA000650C0E94C827C0E08C2F0E94AE0D892B93
:104FB00029F4CF5FC430C1F780E001C081E0CF9118
:104FC00008950E945C2180E00E9430050E94562DC9
:104FD0000E943F1B0C94AE0A1F920F920FB60F92C5
:104FE00011248F939F93AF93BF9380913E048111BF
:104FF00013C080913F0490914004A0914104B0916E
:1050000042044196A11DB11D80933F04909340043A
:10501000A0934104B0934204BF91AF919F918F91AF
:105020000F900FBE0F901F90189582E084BD93E003
:1050300095BD9AEF97BD80936E0008952FB7F894B1
:1050400080913F0490914004A0914104B0914204AA
:105050002FBF0895CF92DF92EF92FF920F931F938D
:105060002FB7F89440913F0450914004609141045F
:10507000709142042FBF6A017B01EE24FF248C0152
:1050800020E030E0C016D106E206F30610F44150ED
:1050900051099A01281B390BC9011F910F91FF90EB
:1050A000EF90DF90CF9008951F920F920FB60F925E
:1050B00011248F939F93AF93BF9380913F0490915E
:1050C0004004A0914104B09142040196A11DB11D7C
:1050D00080933F0490934004A0934104B093420412
:1050E000BF91AF919F918F910F900FBE0F901F9026
:1050F00018950E943C18F8942FEF87EA91E621500A
:1051000080409040E1F700C0000087E090EBDC01B8
:105110008093690490936A04A0936B04B0936C0429
:105120009CE088E10FB6F894A895809360000FBECC
:1051300090936000FFCF0E94DA28811102C00E9484
:10514000B6280E94E52880933D040E94F2288093AF
:10515000670487FB882780F9809385020E94E928ED
:10516000682F70E080E090E00C9418256DEE7EEFE3
:1051700080E090E00E94093260E082E090E00E94CE
:10518000F73160E083E090E00E94F73160E084E076
:1051900090E00E94F73160E085E090E00E94F731F6
:1051A00060E086E090E00E94F7316FEF87E090E0EA
:1051B0000C94F73180E090E00E94F13121E08D3EC7
:1051C0009E4F09F020E0822F089582E090E00C9439
:1051D000E93183E090E00C94E931682F83E090E0BE
:1051E0000C94F73184E090E00C94E931682F84E06E
:1051F00090E00C94F73186E090E00C94E931682F50
:1052000086E090E00C94F73187E090E00C94E9316F
:10521000682F87E090E00C94F7318091450480FF7F
:105220000BC060918B0285E0689FB00111247595D9
:105230006795759567952BC081FF09C060918B02BA
:1052400085E0689FB00111247595679520C082FFA5
:1052500007C060918B0285E0689FB001112417C0E0
:10526000909146049923D1F060918A02961788F7AD
:1052700020918B0285E0289F90011124929FA0012C
:10528000939F500D112470E0CA010E94CF31603805
:10529000710540F46115710539F002C065E070E0F8
:1052A000862F08958FE7089581E008958091450441
:1052B00080FF08C06091890270E0759567957595CB
:1052C000679521C081FF06C06091890270E07595E5
:1052D000679519C082FF04C06091890270E010C018
:1052E000909146049923C1F0609188029617A0F727
:1052F00080918902899FC001112470E00E94CF3102
:105300006038710528F46115710521F0862F089524
:105310008FE7089581E0089561E070E0F4CF803F69
:1053200021F40E940D29819504C0813F29F40E9437
:105330000D29809349040895823F21F40E940D298C
:10534000819504C0833F29F40E940D29809348046D
:105350000895893F19F40E94562905C08A3F31F407
:105360000E945629819580934A0408958B3F21F429
:105370000E945629819504C08C3F29F40E94562929
:1053800080934B040895843F21F480914704816009
:1053900017C0853F21F480914704826011C0863F89
:1053A00021F48091470484600BC0873F21F48091F1
:1053B0004704886005C0883F31F4809147048061CC
:1053C0008093470408958D3F21F4809145048160C6
:1053D0000BC08E3F21F480914504826005C08F3F51
:1053E00029F4809145048460809345040895803FAA
:1053F00039F48091490487FF6CC01092490469C058
:10540000813F29F4809149041816BCF362C0909141
:105410004804823F29F497FF5CC01092480459C0A9
:10542000833F19F41916CCF354C0893F41F480919D
:105430004A0418160CF04DC010924A044AC08A3F24
:1054400029F480914A0487FF44C0F6CF8B3F39F49A
:1054500080914B0487FF3DC010924B043AC08C3FB3
:1054600029F480914B041816BCF333C0843F21F417
:10547000809147048E7F17C0853F21F480914704B7
:105480008D7F11C0863F21F4809147048B7F0BC034
:10549000873F21F480914704877F05C0883F31F41E
:1054A000809147048F7E8093470413C08D3F21F481
:1054B000809145048E7F0BC08E3F21F4809145047E
:1054C0008D7F05C08F3F29F4809145048B7F8093A9
:1054D00045048091480481110EC0809149048111D6
:1054E0000AC080914A04811106C080914B04811149
:1054F00002C010924604089587E494E00E94561B6F
:105500000E941E28909344048093430408951F939F
:10551000CF93DF9380914304909144040E942A2802
:10552000AC0190914604992321F020918C0230E047
:1055300006C020918D028AE0289F90011124421715
:10554000530708F486C080914804C0914904D09163
:105550004A0410914B04811107C0C11176C0D111CA
:1055600074C0111172C075C09F3F19F09F5F909376
:105570004604181624F40E940D2980934804809153
:10558000480487FF05C00E940D2981958093480437
:105590001C1624F40E940D2980934904809149042B
:1055A00087FF05C00E940D29819580934904609171
:1055B0004804662339F1C0914904CC2319F17727B7
:1055C00067FD7095872F972F0E94F12E23E333E319
:1055D00043E35FE30E9401300E94BE2E60934804C3
:1055E0006C2F772767FD7095872F972F0E94F12EDC
:1055F00023E333E343E35FE30E9401300E94BE2EC6
:10560000609349041D1624F40E94562980934A048D
:1056100080914A0487FF05C00E9456298195809396
:105620004A04111624F40E94562980934B04809159
:105630004B0487FF05C00E945629819580934B0437
:10564000DF91CF911F910C947C2A9F3F09F08ECF60
:1056500096CFDF91CF911F910895E7E4F4E085E0C4
:10566000DF011D928A95E9F71092460410924504D5
:105670000895833081F128F4813059F08230D1F0DF
:105680000895853009F449C0B8F1863009F456C050
:10569000089580918D02262F30E0280F311D2F3F75
:1056A000310524F4680F60938D0208958FEF809385
:1056B0008D02089580918C02262F30E0280F311D35
:1056C0002F3F310524F4680F60938C0208958FEF0B
:1056D00080938C02089580918B02262F30E0280F52
:1056E000311D2F3F310524F4680F60938B0208951C
:1056F0008FEF80938B02089580918A02262F30E0ED
:10570000280F311D2F3F310524F4680F60938A0262
:1057100008958FEF80938A02089580918902262F41
:1057200030E0280F311D2F3F310524F4680F6093BE
:10573000890208958FEF80938902089580918802ED
:10574000262F30E0280F311D2F3F310524F4680F3C
:105750006093880208958FEF8093880208958330C4
:1057600011F128F4813049F0823091F008958530AC
:1057700081F120F18630C1F1089580918D02681782
:1057800020F4861B80938D02089510928D02089557
:1057900080918C02681720F4861B80938C020895F8
:1057A00010928C02089580918B02681720F4861B5A
:1057B00080938B02089510928B02089580918A0243
:1057C000681720F4861B80938A02089510928A023B
:1057D000089580918902681720F4861B80938902BE
:1057E000089510928902089580918802681720F424
:1057F000861B8093880208951092880208950F9363
:105800001F93873208F048C08E3108F094C0803171
:1058100009F47EC008F5873009F468C068F4863062
:1058200009F0A4C080913D04817F8E7F80933D0468
:1058300081E080934D049BC08B3009F490C08E3082
:1058400009F094C080913D0482FB222720F991E069
:10585000922790FB82F965C0863109F480C060F41C
:10586000813109F083C00E945C219091850281E022
:1058700089278093850273C0893109F470C08B3108
:1058800009F074C080913D0481FB222720F991E04A
:10589000922790FB81F945C0883309F460C050F429
:1058A000893209F45EC0853309F45BC0873209F49C
:1058B00058C05CC0833409F454C028F48A3308F417
:1058C00055C0895339C0883409F050C00E945C210A
:1058D0000E946C060FEF13ED20E3015010402040B2
:1058E000E1F700C000000E94792839C090913D0482
:1058F000892F8095817080FB90F929F096609860DF
:1059000090933D0434C0997F977F90933D0427C0C6
:1059100080913D0483FB222720F991E0922790FBA0
:1059200083F980933D049923D1F080913D048160F7
:1059300080933D0414C08D5141E050E060E070E080
:105940008A019B0104C0000F111F221F331F8A957B
:10595000D2F7C901B8010E9418250E945C2181E09C
:1059600006C061E070E080E090E0F5CF80E01F913C
:105970000F91089580E0089580E00895CF93C82F97
:1059800080914D04813069F018F08230C9F184C0F3
:10599000E0918602F09187028081823209F07EC018
:1059A00007C0E0918602F09187028081823261F423
:1059B0008C2F0E94BA2C811104C08C2F0E94FF2BC7
:1059C0001DC081E090E01AC08C2F0E94BC2C811178
:1059D00014C0C43179F048F4CB3079F0C03109F00B
:1059E00061C082E080934D0408C0C93219F0C83309
:1059F00021F058C010924D0455C081E0817054C010
:105A0000C93291F120F5C43179F1B0F4C73009F011
:105A100047C08EE180938D0282E380938C028AE0FE
:105A200080938B0284E180938A0288E080938902CC
:105A300088E28093880234C0CE51C63088F5EC2FBE
:105A4000F0E0E85AFC4F808180934C0429C0CE34AA
:105A5000E9F020F4CB3421F56AE013C0C13579F0C8
:105A6000C235F1F461E00DC080914C04882319F037
:105A700010924C0415C081E080934D0415C061E084
:105A800006C080914C040E94392B0AC06AE08091C4
:105A90004C040E94AF2B04C010924D0480E004C05F
:105AA00081E002C080E0AACFCF9108950E94DA2859
:105AB000811102C00E94B6280E94FB2880936804CE
:105AC00080FF02C0869501C080E00C943005809173
:105AD0006804982F9695292F30E0233031054CF437
:105AE0009F5F990F8170892B8160809368040E9469
:105AF000FF288091680486950C9430058091680495
:105B0000982F969591F09158990F8170892B8093D9
:105B100068048E7F91E009F490E08091680490FB26
:105B200080F9809368040E94FF288091680486951C
:105B30000C94300580916804982F909590FB80F923
:105B4000809368040E94FF288091680480FF02C04F
:105B5000869501C080E00C94300590916804892FEF
:105B600086958F5F8F779170843028F4880F892B0A
:105B70008093680402C090936804809168048E7FCB
:105B800091E009F490E08091680490FB80F98093A3
:105B900068040E94FF288091680486950C94300563
:105BA00020916804922F96958927982F990F822F1C
:105BB0008170892B809368048E7F91E009F490E0D6
:105BC0008091680490FB80F9809368040E94FF280C
:105BD0008091680486950C9430055058BB27AA27FD
:105BE0000ED0D1C1C2D130F0C7D120F031F49F3FE7
:105BF00011F41EF4B7C10EF4E095E7FB9FC1E92F45
:105C0000D3D180F3BA17620773078407950718F09A
:105C100071F49EF5EBC10EF4E0950B2EBA2FA02D7A
:105C20000B01B90190010C01CA01A0011124FF2749
:105C3000591B99F0593F50F4503E68F11A16F04044
:105C4000A22F232F342F4427585FF3CF4695379543
:105C50002795A795F0405395C9F77EF41F16BA0B08
:105C6000620B730B840BBAF09150A1F0FF0FBB1FB6
:105C7000661F771F881FC2F70EC0BA0F621F731FFF
:105C8000841F48F4879577956795B795F7959E3F5C
:105C900008F0B3CF9395880F08F09927EE0F9795EA
:105CA0008795089527D108F481E008950CD06BC141
:105CB00063D140F05AD130F021F45F3F19F03EC17A
:105CC000511195C14FC170D198F39923C9F3552350
:105CD000B1F3951B550BBB27AA27621773078407DF
:105CE00038F09F5F5F4F220F331F441FAA1FA9F395
:105CF00033D00E2E3AF0E0E830D091505040E69587
:105D0000001CCAF729D0FE2F27D0660F771F881FE7
:105D1000BB1F261737074807AB07B0E809F0BB0BD6
:105D2000802DBF01FF2793585F4F2AF09E3F5105FA
:105D300068F004C15CC15F3FECF3983EDCF38695EC
:105D400077956795B795F7959F5FC9F7880F911D70
:105D50009695879597F90895E1E0660F771F881F5C
:105D6000BB1F621773078407BA0720F0621B730B0F
:105D7000840BBA0BEE1F88F7E095089504D0689461
:105D8000B11135C1089518D188F09F5790F0B92FFF
:105D90009927B751A0F0D1F0660F771F881F991F80
:105DA0001AF0BA95C9F712C0B13081F01FD1B1E035
:105DB00008951CC1672F782F8827B85F39F0B93F45
:105DC000CCF3869577956795B395D9F73EF4909582
:105DD0008095709561957F4F8F4F9F4F0895E89400
:105DE00009C097FB3EF490958095709561957F4F23
:105DF0008F4F9F4F9923A9F0F92F96E9BB279395D1
:105E0000F695879577956795B795F111F8CFFAF4E0
:105E1000BB0F11F460FF1BC06F5F7F4F8F4F9F4F11
:105E200016C0882311F096E911C0772321F09EE86F
:105E3000872F762F05C0662371F096E8862F70E0D5
:105E400060E02AF09A95660F771F881FDAF7880FAF
:105E50009695879597F9089588D018F011F08CD011
:105E600038F480C0C4C0E92F9FD0B0F35523C9F3E4
:105E7000E7FB6217730784079507A8F199F3E92FE9
:105E8000FF2788232AF03197660F771F881FDAF7DC
:105E9000952F5527442332F091505040220F331F45
:105EA000441FD2F7BB27E91BF50B621B730B840B56
:105EB000B109C1F222F4620F731F841FB11D319723
:105EC0002AF0660F771F881FBB1FEFCF91505040FD
:105ED0005AF041F0882332F0660F771F881F9150E7
:105EE0005040C1F7939530C08695779567959F5F31
:105EF000D9F7F8CF990F0008550FAA0BE0E8FEEF8D
:105F000016161706E807F907C0F012161306E4077D
:105F1000F50798F0621B730B840B950B39F40A2676
:105F200061F0232B242B252B21F408950A2609F454
:105F3000A140A6958FEF811D811D089597F99F6758
:105F400080E870E060E008959F3F31F0915020F4C8
:105F5000879577956795B795880F911D9695879545
:105F600097F908959FEF80EC089500240A9416167F
:105F7000170618060906089500240A941216130637
:105F8000140605060895092E0394000C11F48823C5
:105F900052F0BB0F40F4BF2B11F460FF04C06F5FE1
:105FA0007F4F8F4F9F4F089557FD9058440F551FB7
:105FB00059F05F3F71F04795880F97FB991F61F08B
:105FC0009F3F79F087950895121613061406551F02
:105FD000F2CF4695F1DF08C0161617061806991F6E
:105FE000F1CF86957105610508940895E894BB2763
:105FF00066277727CB0197F908957CDF08F48FEFA8
:1060000008950BD0C0CFB1DF28F0B6DF18F095238C
:1060100009F094CFA7CF1124EACFC6DFA0F3959F54
:10602000D1F3950F50E0551F629FF001729FBB277F
:10603000F00DB11D639FAA27F00DB11DAA1F649F2B
:106040006627B00DA11D661F829F2227B00DA11DDE
:10605000621F739FB00DA11D621F839FA00D611D64
:10606000221F749F3327A00D611D231F849F600D85
:10607000211D822F762F6A2F11249F5750408AF0BE
:10608000E1F088234AF0EE0FFF1FBB1F661F771F4A
:10609000881F91505040A9F79E3F510570F04ECF98
:1060A000A6CF5F3FECF3983EDCF386957795679536
:1060B000B795F795E7959F5FC1F7FE2B880F911D68
:1060C0009695879597F90895FA01EE0FFF1F309680
:1060D0002105310599F16115710561F48038BFE33F
:1060E0009B0749F168949038810561F08038BFEFD3
:1060F0009B0741F0992342F5FF3FE105310521055A
:1061000011F1E8940894E795D901AA2329F4AB2F5B
:10611000BE2FF85FD0F310C0FF5F70F4A695E0F7D4
:10612000F73950F019F0FF3A38F49F779F930CD06D
:106130000F9007FC905808953EF014CF60E070E097
:1061400080E89FE308954FE79F775F934F933F93D6
:106150002F939ED02F913F914F915F9152DF05C0B9
:1061600019F40EF0EBCE42CFFDCE26DFC8F3963801
:10617000C0F707F80F92E8942BE33AEA48EB5FE7A1
:106180004EDF0F920F920F924DB75EB70F92C0D0B5
:10619000ECEFF0E016D04F915F91EF91FF91E59514
:1061A000EE1FFF1F49F0FE57E0684427EE0F441F23
:1061B000FA95E1F74195550B32D00F9007FE26C0B6
:1061C0000895DF93CF931F930F93FF92EF92DF9287
:1061D0007B018C01689405C0DA2EEF011EDFFE0101
:1061E000E894A5912591359145915591AEF3EF0134
:1061F00006DDFE019701A801DA9479F7DF90EF90B0
:10620000FF900F911F91CF91DF9108959B01AC01F9
:1062100060E070E080E89FE349CD90CE95CECCDE83
:10622000E8F39923D9F3940F511DBBF391505040DB
:1062300094F059F0882332F0660F771F881F915031
:106240005040C1F79E3F510544F7880F911D969528
:10625000879597F908955F3FACF0983E9CF0BB2777
:10626000869577956795B79508F4B1609395C1F7D2
:10627000BB0F58F711F460FFE8CF6F5F7F4F8F4F70
:106280009F4FE3CFB4CE0EF05FCE6CCE689456CE67
:1062900093DEC8F39923D1F3C6F3DF93CF931F9313
:1062A0000F93FF92C92FDD2788232AF02197660FCD
:1062B000771F881FDAF720E030E040E85FEB9FE3CC
:1062C000883920F0803E30F021968F7787DCE4E239
:1062D000F1E003C083DCE1E5F1E073DF8B01BE0197
:1062E000EC01FB2E6F5771097595771F880B990B81
:1062F00078DD28E132E741E35FE38FDEAF2D9801DF
:10630000AE01FF900F911F91CF91DF9178DC3BCED2
:10631000FA01DC01AA0FBB1F9B01AC01BF5728F497
:1063200022273327442750781FC0B75188F4AB2F5A
:106330000024469537952795011CA395D2F300209C
:1063400069F0220F331F441FB395DAF30DD045CC0B
:1063500061307105A0E88A07B94630F49B01AC01B1
:106360006627772788279078309621F0208331831D
:10637000428353830895AA1BBB1B51E107C0AA1F88
:10638000BB1FA617B70710F0A61BB70B881F991FD6
:106390005A95A9F780959095BC01CD01089597FB7A
:1063A000072E16F4009407D077FD09D00E94BB3168
:1063B00007FC05D03EF4909581959F4F0895709508
:1063C00061957F4F0895EE0FFF1F0590F491E02D2A
:1063D0000994F999FECF92BD81BDF89A992780B5AD
:1063E0000895A8E1B0E042E050E00C941132262F6D
:1063F000F999FECF92BD81BDF89A019700B40216BB
:1064000039F01FBA20BD0FB6F894FA9AF99A0FBE68
:1064100008950196272F0E94F8310C94F731DC0182
:10642000CB01FC01F999FECF06C0F2BDE1BDF89A9F
:10643000319600B40D9241505040B8F70895F89449
:02644000FFCF8C
:106442000C52D02445000000410000DC4400000052
:106452004152D0A4440000404100005C44000000CE
:106462004148F17644000000415C978A44000000F4
:10647200411FD592440000004152D0A444000000C4
:10648200415CFFB844000000410AA7CF440000006D
:10649200410000DC44000000410AA7CF4400000094
:1064A200410000DC440000004100000000000080C8
:1064B2004000005C450000404100000000000080F8
:1064C2004052D02445000040410AA7CF44000000BA
:1064D200410000DC44000000410000000000008098
:1064E2004052D024450000404100000000000080DE
:1064F2004000005C45000040410AA7CF4400000074
:10650200410000DC44000000410000000000008067
:106512004052D024450000404100000000000080AD
:10652200400AA74F45000040410AA7CF440000009F
:10653200410000DC44000000410000000000008037
:106542004052D024450000004100000000000080BD
:10655200405CFF3845000000410000000000008060
:106562004052D02445000000410AA7CF4400000059
:10657200410000DC440000004100000000000080F7
:106582004052D024450000804153D02445000040B1
:106592004160970A450000004154D0A44400000025
:1065A200410000DC440000004160970A450000A061
:1065B20041050000003F0000C8424314D114AE144C
:1065C2007A14461401012A042808140A321E000013
:1065D200020004000500070009000B000C000E0079
:1065E2001000110013001500170018001A001C00FB
:1065F2001D001F002100230024002600280029007E
:106602002B002D002F0030003200340035003700FF
:1066120039003B0040004500250026006100600073
:1066220020003700640065006600670044004600F1
:10663200240047003149803F5D8B803FF8BF803F97
:10664200CAE1803F73ED803FCAE1803FF8BF803FDF
:106652005D8B803F3149803F0000803FF16D7F3F7D
:1066620075EA7E3F4C827E3F833F7E3F84287E3F99
:10667200833F7E3F4C827E3F75EA7E3FF16D7F3FD6
:106682000000803F3F4D363975092809F208B908E4
:106692004C0865087E0897080102030405060708EE
:0266A2000900ED
:00000001FF
